:10000000AED4DE13AF3412AF3411AF34AF80AE884C
:10001000AC99AFA1E5E253E3F3AFA9BDFDBFF8AEE4
:10002000D322422F4BDA501D9BDA511DAE889BDA4A
:100030005C0B1D9BDA5D0B1DD9BFD82D1ED738ACCC
:10004000A686C087C00F1EACA62D4BDA150B4E9BA3
:10005000DA150B4FAE63EB9B82DCAF80514D504CF9
:10006000AC99BF0580958195BFF8AFA1EDDEBFF8D3
:10007000AEFFAF1E4D40AEFFAF1E4D4C404D0E5675
:100080007C46577D473FAED4AF292349AE884D45C6
:100090004C442746DDBDAF7E0E440A44450A45ED7B
:1000A0005ADDAFBD58DDB1AF7E8667DDB9AF7EAF3B
:1000B00080AFA1E5428973AFA9BD75AED5AF29BFA9
:1000C000F8AED5AEFFDFC5AE63E33CD7FFAD8F5CC6
:1000D000E32A5DEB010F6C410C2F6D42AD8FAC0834
:1000E0005C1BAD8FAC085D1A4C19AD8FAD8FAE9611
:1000F00081138213AD8F57E30356EB3CBF05BFF866
:00000001FF
